:0300000002347E49
:0C347E0078FFE4F6D8FD75816A0234C5C1
:100EE20020000A3C2E2E2E3E004950436F6E6E6546
:100EF20063745245510A004950436F6E6E656374C4
:100F0200000A49504E6F41434B210A003E432C5682
:100F12002C43432CC0E4E0EFF2E5F020D1E8EDEA07
:100F2200EEEC49500A003E432C4D41432C25303211
:100F320062583A25303262583A25303262583A25A0
:100F4200303262583A25303262583A25303262588D
:100F52002C4D414320E0E4F0E5F10A003E432C56DB
:100F620045522C20332E3220EEF220257320257399
:100F72002CC2E5F0F1E8FF20495020ECEEE4F3EB5F
:100F8200FF0A004A756E2032352032303039003186
:100F9200333A32343A3231003E432C4C442C5052D4
:100FA2004F473A20202020202020202020202020CF
:100FB200202020202020202020202020202020202F
:100FC200202020202020202020202020202020201F
:100FD200202020202020202020202020202020200F
:100FE20020202020202020202CC4E0F2E020EFF05E
:100FF200EEF8E8E2EAE828F4E0E9EB290A003E2A02
:101002002C312CCEF1EDEEE2EDFBE520EFE0F0E04D
:10101200ECE5F2F0FB20F1E5F2E5E2EEE3EE20E8AA
:10102200EDF2E5F0F4E5E9F1E00A003E412C413051
:10103200312C2562752E2562752E2562752E25624C
:10104200752C495020E0E4F0E5F120E0E4E0EFF215
:10105200E5F0E00A003E412C4130322C2562752E2B
:101062002562752E2562752E2562752C495020E069
:10107200E4F0E5F120EEF1ED2E20F1E5F0E2E5F00D
:10108200E00A003E412C4130332C2562752E256248
:10109200752E2562752E2562752C495020E0E4F0EC
:1010A200E5F120F0E5E72E20F1E5F0E2E5F0E00AD7
:1010B200003E412C4130342C2562752E2562752E5E
:1010C2002562752E2562752CCCE0F1EAE020F1E56F
:1010D200F2E80A003E412C4130352C2562752E255E
:1010E20062752E2562752E2562752CD8EBFEE70AF5
:1010F200003E2A2C312CC4EEEF2E20EFE0F0E0EC83
:10110200E5F2F0FB20F1E5F2E5E2EEE3EE20E8EDB8
:10111200F2E5F0F4E5E9F1E00A003E422C53303109
:101122002C2562752CC6E4E0F2FC20E7E0EFF0EE3D
:10113200F1E020F1EEE5E4E8EDE5EDE8FF20EEF286
:1011420020F1E5F0E2E5F0E00A003E422C533032B5
:101152002C2562752CCEE1ECE5ED20F120F1E5F0D5
:10116200E2E5F0EEEC20E1E5E720EAE2E8F2E0ED8C
:10117200F6E8E90A003E422C5330332C2562752CE6
:10118200CFE5F0E5E7E0EFF3F1EA20EFF0E820EF5A
:10119200EEF2E5F0E520F1E2FFE7E820F120F1E5EB
:1011A200F0E2E5F0EEEC0A003E454E440A000A4445
:1011B200756D7058202020202030302030312030B2
:1011C2003220303320303420303520303620303752
:1011D2002030382030392030412030422030432026
:1011E2003044203045203046000A3A003A20000AB6
:1011F200000A44756D7044202020202030302030B9
:101202003120303220303320303420303520303617
:1012120020303720303820303920304120304220F1
:101222003043203044203045203046004572722041
:101232006B657900526420656570726F6D0A0052A9
:1012420064204D454D0A00526420436F64650A00D4
:10125200577269746520436F64650A00446562755C
:10126200674950204F4E0A00446562756749502015
:101272004F46460A00446562756755736572204F92
:101282006E0A00446562756755736572204F464663
:101292000A0044656275674D7367204F6E0A004409
:1012A200656275674D7367204F46460A00436F6E4D
:1012B200666967206C6F636B210A0057722065654F
:1012C20070726F6D0A0020536176652065657072D9
:1012D2006F6D210A00457272204D414321004C6F0F
:1012E20061643E3E002A003C4130313D003C4130C9
:1012F200323D003C4130333D003C4130343D003C06
:101302004130353D003C21003C5330313D003C53DF
:1013120030323D003C5330333D003C5330353D00CC
:061322003C5330363D0093
:063DC70001670001650028
:103E2D00C28E438910E4F58B758DB8D2ABD28E223C
:03001B000233EEBF
:1033EE00C0E0C083C082C0D0C28E758B00758DB810
:1033FE0020060675A61E75A6E10565D202E5676074
:10340E00020567E566D3940140021566056AE56A12
:10341E00540F7048D20EE56A543F7012D200906677
:10342E008BE0600A04F0E0D394B44002D2069066BA
:10343E0086E0600204F0906104E0600214F0906691
:10344E008CE0D394014003E014F03005020568E5EA
:10345E0069D394644004D20680020569E564D3946E
:10346E000140021564D28ED0D0D082D083D0E0320B
:10087900C291C290D2B5C20B7D027C007F07123DA6
:10088900AA8F25E525646060097D017F60123D45D9
:10089900D20BE4FDFC7F0B123DAA8F25E52530E63E
:1008A900097D04E4FF123D69D20B7D017C007F07BD
:1008B900123DAA8F25E5257008FD7FFF123D45D21F
:1008C9000B300B03126000C288C2A8C2AA75890046
:1008D9001237A690633EE0B4FA06A3E064CE607BCB
:1008E900E4F52574362525F582E43463F583E4F0CF
:1008F9000525E525B443EC90633E74FAF0A374CE64
:10090900F0A374CCF0906344740AF0E4A3F0A30458
:10091900F0A3F090633A74FFF0A3F0A3F0E4A3F01E
:10092900906355740AF0E4F525E5252401FFE433C5
:10093900FE74362525F582E43463F583E0FD123D26
:10094900210525E525C3944340DFE4F5A775A61ED7
:1009590075A6E1907FF0F0A3F080FE9063497403DF
:10096900F0A374CCF0E4906348F0123057C2B5128A
:100979003DE3C206123A92D20BC20DC20C906576C3
:100989007408F09062B47424F0E4A3F090633EE03C
:100999009062B6F090633FE09062B7F0906340E0F8
:1009A9009062B8F0906341E09062B9F0906342E0E0
:1009B9009062BAF0906343E09062BBF0756601E41F
:1009C900906577F0C207C208C209C20A200B18AFA6
:1009D90025FE7D03122E9BE4FF12333E7E0E7FE23D
:1009E900E4FBFDFC122AA790668BE060037401F01A
:1009F900E4906104F0F568906575F0F569123E2D93
:100A090075A70775A61E75A6E1D2AFE4F5699061D1
:100A190004E0700312168490668CE06401701D90E6
:100A290080007410F09080A874FFF0A3F0A3F0A3E5
:100A3900F0E490668CF0D20BC20CC20D908008E0F5
:100A4900F52530E405D2077410F0E52530E508D224
:100A5900099080087420F0E52530E608D2089080D6
:100A6900087440F0E568C394034019908002E4F0EB
:100A7900908001F0908000F0E56894064006E4F566
:100A890068123A929080A0E0700312390D9080B8F4
:100A9900E070031238249080D0E07003123A369047
:100AA9008000E07013300710122BAE906331EFF025
:100AB900D394004003120036908002E070069080C3
:100AC90000E06005D205020A14C205E4F5689061E8
:100AD90004E06003020A14200B12906578E0600CB0
:100AE9007E0E7FE4122DB3E4906578F0300912127E
:100AF900254E906331EFF0D394004005E0FF1200DA
:100B090032200803020C8A1223C7906331EFF07078
:100B190003020A14906375E054BF247F7003020B2B
:100B2900F3147003020BCB24026003020C2C200B7C
:100B3900077E0E7FEB122DB3200F03020C8A906300
:100B49004DE07006906351E06067906682E0FF9027
:100B5900634DE0B50724906683E0FE90634EE0B5EF
:100B69000618906684E0FE90634FE0B5060C906627
:100B790085E0FE906350E06E6037906351E06F60EE
:100B890003020C8A906683E0FF906352E06F600372
:100B9900020C8A906684E0FF906353E06F60030261
:100BA9000C8A906685E0FF906354E06F6003020C45
:100BB9008AC2039065777401F0123E53756601028B
:100BC9000C8A90668BE060037401F090667AE0FF0E
:100BD900906377E06F6003020C8A90667AE004F014
:100BE900E4F566906575F0020C8A300303020C8AFD
:100BF900906344E07003020A14906355740AF0127A
:100C09003B45D203E4F566906575F090668604F07D
:100C1900E4906679F0A3F0200B677E0E7FF9122D20
:100C2900B3805E90668BE060037401F030035290EC
:100C39006375E020E74B906377E0FF906679E0FE0B
:100C49006F600D906681E07007EE146F703380134A
:100C5900906679E004F0906331E0FFD39404400397
:100C690012389E9060007482F0A37401F09063774B
:100C7900E0906002F07E607F007D03123591020AE8
:100C890014200303020DA2E5667068122989EF603A
:100C9900237E647F75906476E02404FD123591907B
:100CA9006681E07009906355E0F566020A14E4F57F
:100CB90066020A14906686E0D3943C4036906681B9
:100CC900E0703090668604F01231D8E4906475F0D3
:100CD900A37412F090667AE0906477F0A374FDF043
:100CE90090610563A20190647963A2017F12121FCA
:100CF90068809E123E488F25E525B4011590600055
:100D09007483F0E4A3F07E607F007D0212359102C6
:100D19000A14E525D39401401C9060007483F0A364
:100D29007401F0E52524FEA3F07E607F007D0312A7
:100D39003591020A14E56664016003020A1490659C
:100D490075E004F0200B077E0F7F03122DB390632B
:100D590055E0C394C85004E02432F0906575E0C3AF
:100D69009405400DC203E4906577F0123E53020AE0
:100D7900147C667D82906349E0FAA3E0FB7F02124E
:100D890037227E647F75906476E02404FD123591E4
:100D9900906355E0F566020A14E566640160030292
:100DA9000A14906577E014604624FE6042147003CB
:100DB900020E9524046003020A14E4F568200F1357
:100DC9009065777404F0906575E05401F0756601DB
:100DD900020A149080027410F0E4906577F090652F
:100DE9007504F07566FA90668274FFF0020A149031
:100DF9006682E07003020E7F9064757480F09064DF
:100E0900777401F0E4A3F0A304F0A37430F0A374A1
:100E19007BF0E4F525747C2525F582E43464F583BB
:100E2900747DF0747D2525F582E43464F583E4F05E
:100E3900E5252407906476F07C667D82906349E01D
:100E4900FAA3E0FB7F021237227E647F75E5252431
:100E590009FD123591906681E0601B123B45D20372
:100E6900E4F566906575F090668604F0E49066791D
:100E7900F0A3F0020A14300F07E4906577F08006BA
:100E89009065777404F07566FA020A14908002740A
:100E990010F0756605906575E06401FFF09065775F
:100EA9007401F0EF7019906351E06013FCA3E0FD49
:100EB900A3E0FEA3E0FF906682121D4F020A149080
:100EC900634DE0FCA3E0FDA3E0FEA3E0FF90668292
:080ED900121D4F020A1480FEF5
:010EE10022EE
:10003600906376E0B444047F0180027F009063758C
:10004600E0B447047E0180027E00EE5F604A906362
:100056003EE0906377F090633FE0906378F09063C2
:1000660040E0906379F0906341E090637AF09063AA
:1000760042E090637BF0906343E090637CF0906392
:10008600767452F09062AE63A2019080A863A201DA
:100096007F06121F6802086F906331E0C394085010
:1000A6000302087890633EE0FF906377E06F600399
:1000B60002087890633FE0FF906378E06F60030288
:1000C6000878906340E0FF906379E06F6003020870
:1000D60078906341E0FF90637AE06F6003020878EE
:1000E600906342E0FF90637BE06F600302087890C4
:1000F6006343E0FF90637CE06F60030208789063DF
:1001060076E06444701A9080A8E0B4FF139062AE63
:1001160063A2019080A863A2017F06121F68801067
:100126009062B2E09080ACF09062B3E09080ADF067
:1001360090668BE060037401F090668C7464F090B6
:1001460063767452F0906375E0646D600302027921
:100156007BFF7A0F790E12138A7BFF7A0F7928902C
:10016600633EE0F52EA3E0F52FA3E0F530A3E0F51E
:1001760031A3E0F532A3E0F53312138A752EFF752D
:100186002F0F7530857531FF75320F7533917BFFF3
:100196007A0F795E12138A7BFF7A0F799A12138A85
:1001A6007BFF7A10790012138A7BFF7A10792D90E3
:1001B6006344E0F52EA3E0F52FA3E0F530A3E0F5C8
:1001C6003112138A7BFF7A10795790634DE0F52E32
:1001D600A3E0F52FA3E0F530A3E0F53112138A7BF7
:1001E600FF7A107985906351E0F52EA3E0F52FA3F1
:1001F600E0F530A3E0F53112138A7BFF7A1079B36C
:1002060090633AE0F52EA3E0F52FA3E0F530A3E0E6
:10021600F53112138A7BFF7A1079D6906336E0F5B2
:100226002EA3E0F52FA3E0F530A3E0F53112138AF3
:100236007BFF7A1079F312138A7BFF7A11791CA25D
:100246000FE433F52E12138A7BFF7A11794C9066F0
:1002560081E0F52E12138A7BFF7A11797790668BEF
:10026600E0F52E12138A122CB27BFF7A1179AA12AC
:10027600138A22906375E0644C70737E117FB0FB25
:10028600FDFC122AA790637DE0F526A3E0F527E49E
:10029600F529E52690637FF0A3E527F07E117FEB35
:1002A6007C637D7F7B02122AA7E4F5288527828559
:1002B6002683E0FF747F2528F582E43463F583EF17
:1002C600F00527E527700205260528E528B410DC89
:1002D6007E117FEE7C637D7F7B10122AA70529E5C0
:1002E60029C3941040AC7E117FF1122DB322906386
:1002F60075E0646C7060F52A7E117FF3FBFDFC12DD
:100306002AA7E4F529E490637FF0A3E52AF07E119D
:100316007FEB7C637D7F7B02122AA7E4F528A82A5F
:10032600E6FF747F2528F582E43463F583EFF00554
:100336002A0528E528B410E67E117FEE7C637D7FD2
:100346007B10122AA70529E529C3940840B77E1118
:100356007FF1122DB322906375E0644B7061F5282E
:1003660074672528F582E43463F583E060327467A8
:100376002528F582E43463F583E0F4602374672569
:1003860028F582E43463F583E0FF747D2528F58241
:10039600E43463F583E0B507100528E528B408C002
:1003A6009061047432F002086F9063757421F03026
:1003B6000B0302086F7E127F2E122DB302086F9078
:1003C6006375E0B4521A200B077E127F36122DB3E6
:1003D6009063757472F07E637F757D0812350A220C
:1003E600906375E064497045200B077E127F4112C9
:1003F6002DB390637DE0F526A3E0F527E4F5288587
:100406002782852683E0FF747F2528F582E43463FE
:10041600F583EFF00527E527700205260528E52870
:10042600B480DC7E637F757D8A12350A22906375FF
:10043600E064437046200B077E127F49122DB3906D
:10044600637DE0F526A3E0F527E4F5288527828578
:100456002683E493FF747F2528F582E43463F583CD
:10046600EFF00527E527700205260528E528B48064
:10047600DB7E637F757D8A12350A22906375E064A0
:100486005A7053200B077E127F52122DB390637D54
:10049600E0F526A3E0F5277C637D7F7B80AF27AE62
:1004A60026123CC6E4F528852782852683E493FF39
:1004B600747F2528F582E43463F583EFF00527E59C
:1004C60027700205260528E528B480DB7E637F7544
:1004D6007D8A12350A22906375E064446003020542
:1004E6006D90637DE0FF6444700302086FEFB431E2
:1004F6000CC20B7E127F5E122DB302086F90637DD5
:10050600E0B4300CD20B7E127F6A122DB302086F54
:1005160090637DE0B4320CD20C7E127F77122DB33D
:1005260002086F90637DE0B4330CC20C7E127F85A7
:10053600122DB302086F90637DE0B4340CD20D7EA9
:10054600127F94122DB302086F90637DE0B4350CD0
:10055600C20D7E127FA1122DB302086F90637DE05B
:10056600FF12001E02086F906104E07013200B0753
:100576007E127FAF122DB39063757421F002086F5F
:100586009061047432F0906375E0FFB45104C2AF19
:1005960080FEEF64577045200B077E127FBD122D3B
:1005A600B390637EE0906331F0E4F528906331E028
:1005B600FFE528C39F400302086F747F2528F58254
:1005C600E43463F583E0FF90637DE0252824ADF5F0
:1005D60082E43461F583EFF0052880D0906375E0FE
:1005E60064536003020690200B077E127FC8122D0B
:1005F600B390633EE0FF9061B6E06F703C90633F5E
:10060600E0FF9061B7E06F7030906340E0FF90616B
:10061600B8E0B50724906341E0FF9061B9E0B50703
:1006260018906342E0FF9061BAE0B5070C9063430F
:10063600E0FF9061BBE06F60169063757421F03047
:100646000B0302086F7E127FD7122DB302086FE4E8
:10065600F528E4F569AF28FE74AD2528F582E43463
:1006660061F583E0FD123D210528E528C394FE408F
:10067600E1C2AFE4907FF0F0A3F0907FFD74AAF0A2
:10068600A374FFF0A37455F080FE906375E0644F89
:10069600704C90637DE0F526A3E0F527E527452617
:1006A600700A200B077E127FE0122DB3200B077E07
:1006B600127FE7122DB3E4F528747F2528F582E42E
:1006C6003463F583E0852782852683F00527E527B1
:1006D600700205260528E528B480DE02086F9063BF
:1006E60075E0FFB4452190637DE0FDA3E0907FF0C7
:1006F600CDF0A3EDF0C2AF907FFD74AAF0A374FF16
:10070600F0A37455F080FEEF6465600302087890EC
:10071600637DE0FFA3E0907FF0CFF0A3EFF0E4F578
:1007260026F527D3907FF1E09527907FF0E0952678
:100736004020E4F5692527FFE5263401FE8527825A
:10074600852683E0FD123D210527E5277002052653
:1007560080D17E127FE9123618EF4E602012000318
:10076600906344EFF0120003906345EFF01200032C
:10077600906346EFF0120003906347EFF07E127F1E
:10078600EF123618EF4E602012000390634DEFF023
:1007960012000390634EEFF012000390634FEFF0E8
:1007A600120003906350EFF07E127FF5123618EFB9
:1007B6004E6020120003906351EFF0120003906325
:1007C60052EFF0120003906353EFF01200039063B0
:1007D60054EFF07E127FFB123618EF4E60201200A7
:1007E6000390633AEFF012000390633BEFF01200C0
:1007F6000390633CEFF012000390633DEFF07E132D
:100806007F01123618EF4E6020120003906336EF18
:10081600F0120003906337EFF0120003906338EF95
:10082600F0120003906339EFF0E4F528E4F569E58A
:10083600282401FFE433FE74362528F582E4346368
:10084600F583E0FD123D210528E528C3944340DCED
:10085600C2AFE4907FF0F0A3F0907FFD74AAF0A3FE
:1008660074FFF0A37455F080FE7E637F757D0812D9
:02087600350A41
:01087800225D
:103C8E00AE07EEC39430400BEED394395005EE24BC
:103C9E00D0FF22EEC39461400BEED394665005EE36
:103CAE0024A9FF22EEC39441400BEED39446500557
:083CBE00EE24C9FF22AF06222B
:103DFF009062ADE004F070069062ACE004F0906267
:0A3E0F00ACE0FEA3E0FF123D8D229F
:10000300123DFF123C8EEFC454F0FEC006123DFFBA
:08001300123C8ED0E02FFF2209
:1039D900E4906A3CF0123DFF906A3DEFF0C39430E9
:1039E9004018E0FFD394395011906A3CE02405F562
:1039F90082E43461F583EFF08011906A3CE024059C
:103A0900F582E43461F583E4F0800C906A3CE004CB
:103A1900F0E0D3940840BE7531007532007533006B
:0C3A2900E4F5347B017A61790512222358
:013A3500226E
:043618008E2B8F2C3A
:10361C009062ACE4F0A374FFF0123DFFEF606EF427
:10362C00606B852C82852B83E493B507EC752D019B
:10363C00E52C252DF582E4352BF583E4936025905C
:10364C0062ADE0252DFF9062ACE03400FE123D8DA2
:10365C00E52C252DF582E4352BF583E493B5070491
:10366C00052D80CCE52C252DF582E4352BF583E456
:10367C009370A6E52D24FFFFE434FFFE9062ADE0CD
:10368C002FF09062ACE03EF07E007F0122E4FEFF62
:01369C00220B
:103057007E137F07123618EF4E70037F01227E130F
:103067007F0A123618EF4E600C123DFFEF24D02472
:10307700FF920F8002D20F7E137F10123618EF4E89
:10308700600C123DFFEF24D0906681F08005E4903C
:103097006681F07E137F16123618EF4E600C123DD4
:1030A700FFEF24D090668BF08005E490668BF07E6E
:1030B700137F1C123618EF4E600C123DFFEF24D021
:1030C70024FF92018002C20190633E63A2019066D1
:1030D7007B63A2017F06121F6830013B7E137F22AC
:1030E700123618EF4E603012000390667BEFF01235
:1030F700000390667CEFF012000390667DEFF012FC
:10310700000390667EEFF012000390667FEFF012E7
:0A3117000003906680EFF07F0022B5
:103B9A00906576E0C3947C40027F0A906576E0FEE9
:103BAA0004F074B42EF582E43462F583EFF0BF0AB0
:103BBA0027906576E0FF04F074B42FF582E434624E
:103BCA00F583E4F0906576E0FF12369D9065767491
:093BDA0008F09062B5E004F0224D
:103A92009080007480F090633663A201F583F58212
:103AA20063A2017F08121F6890633E63A2019080A7
:103AB2008863A2017F0A121F689080927407F0A3A4
:103AC20074D0F0A37406F0906348E0FF9080B1F0E8
:103AD2009080E1EFF09080957455F0A3F090800013
:0A3AE2007401F090800974F0F022E6
:10390D00908009E04410F09080A0E070609080A15C
:10391D007482F09080A874FFF0A3F0A3F0A3F07F61
:10392D00039080AEEFF0A374CBF09080007402F0A2
:10393D00906A2C121D5B00000000906A2CE09080B4
:10394D0040F0906A2DE0908041F0906A2EE09080DA
:10395D0042F0906A2FE0908043F0A3E4F0A3F0A32F
:0D396D00F0A3F0908018F0A3F0A3F0A3F0F9
:01397A00222A
:103A3600908009E04440F09080D17482F07F03903A
:103A460080DEEFF0A374CCF09080027402F0906AEE
:103A560030121D5B00000000906A30E0908058F044
:103A6600906A31E0908059F0906A32E090805AF086
:103A7600906A33E090805BF0A3E4F0A3F0A3F0A398
:0B3A8600F0908030F0A3F0A3F0A3F05C
:013A91002212
:10382400908009E04420F09080B8E0706C9080B9FA
:103834007482F07F039080C6EFF07FCDA3EFF07F1A
:10384400039080C4EFF0A374CDF09080C074FFF0B7
:10385400A3F0A3F0A3F09080017402F0906A3412F4
:103864001D5B00000000906A34E090804CF0906A88
:1038740035E090804DF0906A36E090804EF0906A8A
:1038840037E090804FF0A3E4F0A3F0A3F0A3F0900E
:093894008024F0A3F0A3F0A3F0DE
:01389D002208
:103722008C268D27A907EAFDE975F018A424ACFFC1
:10373200E5F034808F82F583EDF0EBFDE975F0184A
:10374200A4FFAEF024ACFBEE34808B82F583A3EDB4
:10375200F08527828C83E0FDEF24A8FFEE3480FE03
:103762008F82F583EDF08527828C83A3E08F828E92
:1037720083A3F0852782852683A3A3E0FDE975F064
:1037820018A424A8FFE5F03480FE8F82F583A3A35A
:10379200EDF08527828C83A3A3A3E08F828E83A37F
:0437A200A3A3F022CB
:06350A008D2BAB07AA06A1
:10351000908000E030E5079065787401F022906AB1
:103520002CE0FCA3E0FDA3E0FEA3E0F52F8E2E8DA2
:103530002D8C2CAE02AF038E838F8263A201E52E09
:10354000540744C0F583852F8263A201AF2B121F5D
:10355000DAE4FCFDFEE52F252BF52FEE352EF52EBA
:10356000ED352DF52DEC352CF52C908040E52CF02B
:10357000A3E52DF0A3E52EF0A3E52FF090800074D5
:1035800020F0AF2FAE2EAD2DAC2C906A2C121D4F1B
:013590002218
:063591008D26AB07AA061F
:10359700908002E030E5079065787403F022906A26
:1035A70030E0FCA3E0FDA3E0FEA3E0F52A8E298D21
:1035B700288C27AE02AF038E838F8263A201E52991
:1035C700540744D0F583852A8263A201AF26121FD0
:1035D700DAE4FCFDFEE52A2526F52AEE3529F5294C
:1035E700ED3528F528EC3527F527908058E527F0A5
:1035F700A3E528F0A3E529F0A3E52AF0908002745B
:1036070020F0AF2AAE29AD28AC27906A30121D4FA3
:013617002290
:02333E008F26D8
:10334000908001E030E5099065787402F07F0022FA
:10335000906A34E0FCA3E0FDA3E0FEA3E0F52A8E32
:10336000298D288C2790667B63A201E529540744A8
:10337000C8F583852A8263A2017F06121FF0E52A21
:103380002406F52AE43529F529E43528F528E4351D
:1033900027F52790657963A201E529540744C8F50C
:1033A00083852A8263A201AF26121FF0E4FCFDFE92
:1033B000E52A2526F52AEE3529F529ED3528F528C3
:1033C000EC3527F52790804CE527F0A3E528F0A3FE
:1033D000E529F0A3E52AF09080017420F0AF2AAE31
:0D33E00029AD28AC27906A34121D4FAF268E
:0133ED0022BD
:102BAE009081E0E0F5260526052605260526052654
:102BBE0005260526052605260526908010E0F52912
:102BCE00A3E0F52AA3E0F52BA3E0F52C9081E1E03C
:102BDE00F52605260526052605260526052605269F
:102BEE00052605260526908014E0F52DA3E0F52E8A
:102BFE00A3E0F52FA3E0F530E52FB52B08E530B5B2
:102C0E002C037F0022E4F526E52F540744E0F583DC
:102C1E0085308263A20190637563A2017F08122042
:102C2E002090637763A2019062AE63A2017F0612C9
:102C3E001F68906375E0F527A3E0F528E4F526906C
:102C4E006375E0702AA3E024F8F526E52F540744B7
:102C5E00E0F58385308274082582F582E43583F5AC
:102C6E008363A20190637563A201AF26122020AE8A
:102C7E0027E4FCFDE5302528F530E52F3EF52FED58
:102C8E00352EF52EEC352DF52D908014E52DF0A377
:102C9E00E52EF0A3E52FF0A3E530F0908000744010
:032CAE00F0AF265E
:012CB1002200
:1023C7009081E6E0F526052605260526052605263D
:1023D70005260526052605260526908028E0F529E9
:1023E700A3E0F52AA3E0F52BA3E0F52C9081E7E025
:1023F700F52605260526052605260526052605268E
:1024070005260526052690802CE0F52DA3E0F52E60
:10241700A3E0F52FA3E0F530E4F526E52FB52B0A69
:10242700E530B52C05C208022533E52F540744F0E3
:10243700F58385308263A20190637563A2017F08EB
:10244700122020906375E0F527A3E0F528E52845DD
:102457002770099080027410F07F0022906682E056
:10246700FFF46030906377E06F60030224FA9066B0
:1024770083E0FF906378E06F7079906684E0FF9067
:102487006379E06F706D906685E0FF90637AE06F27
:102497006031805F906377E0906682F0906378E0C8
:1024A700906683F0906379E0906684F090637AE0B9
:1024B700906685F090637BE0FFA3E0906349CFF0DF
:1024C700A3EFF0906375E0702AA3E024F8F526E502
:1024D7002F540744F0F58385308274082582F582EE
:1024E700E43583F58363A20190637563A201AF2688
:1024F700122020AE27E4FCFDE5302528F530E52F36
:102507003EF52FED352EF52EEC352DF52DAF2CAEF6
:102517002BAD2AAC29AB30AA2FA92EA82DD3121D7B
:102527003E40099080027410F07F002290802CE5D5
:102537002DF0A3E52EF0A3E52FF0A3E530F0908072
:06254700027440F0AF2613
:01254D00226B
:10254E009081E3E0F52605260526052605260526B7
:10255E000526052605260526052690801CE0F5296C
:10256E00A3E0F52AA3E0F52BA3E0F52C9081E4E09F
:10257E00F526052605260526052605260526052605
:10258E00052605260526908020E0F52DA3E0F52EE4
:10259E00A3E0F52FA3E0F530E4F526E52FB52B0AE1
:1025AE00E530B52C05C2090226A4E52F540744E8F0
:1025BE00F58385308263A20190600463A2017F0ED1
:1025CE00122036906004E0F527A3E0F52890600C09
:1025DE00E0FFF4604A90667BE0FEEF6E7079A3E058
:1025EE00FF90600DE06F706F90667DE0FF90600E63
:1025FE00E06F706390667EE0FF90600FE06F705743
:10260E0090667FE0FF906010E06F704B906680E008
:10261E00FF906011E06F703FE4906013F0800890BF
:10262E00601374FFF0D2D9906004E0702AA3E02406
:10263E00F2F526E52F540744E8F583853082740EB3
:10264E002582F582E43583F58363A20190600463ED
:10265E00A201AF26122036AE27E4FCFDE530252878
:10266E00F530E52F3EF52FED352EF52EEC352DF50B
:10267E002DAF2CAE2BAD2AAC29AB30AA2FA92EA88C
:10268E002DD3121D3E5006E5284527700990800176
:10269E007410F07F0022908020E52DF0A3E52EF03F
:1026AE00A3E52FF0A3E530F09080017440F0AF2643
:0126BE0022F9
:042DB3008E2B8F2CA8
:102DB700908000E030E5079065787401F022906A12
:102DC7002CE0FCA3E0FDA3E0FEA3E0F5328E318DFD
:102DD700308C2FE532FFE5315407FEE42FF52EEE58
:102DE70034C0F52D852E82F5837423F0052EE52E4C
:102DF7007002052D532DC7F582852D83740AF005C2
:102E07002EE52E7002052D532DC790633E63A20158
:102E1700852D83852E8263A2017F06121FDA740631
:102E2700252EF52EE4352DF52D852B83852C8263F4
:102E3700A201852D83852E8263A201121FBEE4FCA9
:102E4700FDFE906A2CE0F8A3E0F9A3E0FAA3E02FD7
:102E5700FFEE3AFEED39FDEC38FCEF2408FFE43EC7
:102E6700FEE43DFDE43CFC906A2C121D4F906A2C59
:102E7700E0908040F0906A2DE0908041F0906A2EBB
:102E8700E0908042F0906A2FE0908043F0908000BD
:032E97007420F0B4
:012E9A002215
:0A2AA7008E2B8F2C8C2D8D2E8B2F83
:102AB100908000E030E5079065787401F022906A1B
:102AC1002CE0FCA3E0FDA3E0FEA3E0F5358E348D00
:102AD100338C32E535FFE5345407FEE42FF531EE52
:102AE10034C0F530853182F5837423F00531E53149
:102AF100700205305330C7F582853083740AF005C2
:102B010031E531700205305330C790633E63A20155
:102B110085308385318263A2017F06121FDA740634
:102B21002531F531E43530F530852B83852C8263F1
:102B3100A20185308385318263A201121FBE8F36C7
:102B4100EF2531F531E43530F530E52F6017852D6E
:102B510083852E8263A20185308385318263A20140
:102B6100AF2F121FDAE5362408252FF52FFFE4FCDD
:102B7100FDFEE5352FF535EE3534F534ED3533F51C
:102B810033EC3532F532908040E532F0A3E533F095
:102B9100A3E534F0A3E535F09080007420F0AF3563
:0C2BA100AE34AD33AC32906A2C121D4FE4
:012BAD002205
:062F7C008E288F298D2A2A
:102F8200908000E030E5079065787401F022906A45
:102F92002CE0FCA3E0FDA3E0FEA3E0F5308E2F8D34
:102FA2002E8C2DE530FFE52F5407FEE42FF52CEE95
:102FB20034C0F52B852C82F5837423F0052CE52C87
:102FC2007002052B532BC7F582852B83EBF0052C62
:102FD200E52C7002052B532BC790633E63A201853B
:102FE2002B83852C8263A2017F06121FDA740625C9
:102FF2002CF52CE4352BF52B85288385298263A2B9
:1030020001852B83852C8263A201AF2A121FDA74F9
:1030120008252AF52AFFE4FCFDFEE5302FF530EE07
:10302200352FF52FED352EF52EEC352DF52D908023
:1030320040E52DF0A3E52EF0A3E52FF0A3E530F057
:103042009080007420F0AF30AE2FAD2EAC2D906A80
:043052002C121D4FD0
:013056002257
:02369D008F3F5D
:10369F00908000E030E5079065787401F022906A21
:1036AF002CE0FCA3E0FDA3E0FEA3E0F5438E428DEA
:1036BF00418C40E543FFE5425407FEE42FFFEE3413
:1036CF00C09062B463A201F5838F8263A201AF3F02
:1036DF00121FDAE4FCFDFEE543253FF543EE3542CC
:1036EF00F542ED3541F541EC3540F540908040E530
:1036FF0040F0A3E541F0A3E542F0A3E543F090804D
:10370F00007420F0AF43AE42AD41AC40906A2C1232
:02371F001D4F3C
:013721002285
:062E9B008E2E8F2FAB0507
:102EA100908000E030E5079065787401F022906A27
:102EB1002CE0FCA3E0FDA3E0FEA3E0F5358E348D0C
:102EC100338C32E535FFE5345407FEE42FF531EE5E
:102ED10034C0F530853182F5837423F00531E53155
:102EE100700205305330C7F582853083EBF0053130
:102EF100E5317002053090633E63A2018530838520
:102F0100318263A2017F06121FDA74062531F53181
:102F1100E43530F5305330C7E52E85318285308375
:102F2100F00531E531700205305330C7F582853047
:102F310083E52FF00531E531700205305330C7E5E7
:102F410035240AF535E43534F534E43533F533E425
:102F51003532F532908040E532F0A3E533F0A3E558
:102F610034F0A3E535F09080007420F0AF35AE3435
:0A2F7100AD33AC32906A2C121D4FF4
:012F7B002233
:0A3E3D00E4FEEEC39F50030E80F870
:013E47002258
:103D8D00A2AF921EC2AF438E2075D2028F828E8358
:0C3D9D00E0FFE4F5D2538EDFA21E92AFCF
:013DA90022F7
:103D2100E5D220E0FBA2AF921EC2AF43D2028F8246
:103D31008E83EDF075D25063D250A21E92AFE5D2C0
:033D410020E0FB84
:013D4400225C
:1037A600E4FDED2401FFE433FE123D8D74362DF564
:1037B60082E43463F583EFF00DBD3FE6E4FDED24CE
:1037C6007FFFE433FE123D8D742D2DF582E43461C6
:1037D600F583EFF0742D2DF582E43461F583E07006
:1037E6001B742D2DF582E43461F5837420F0742E5C
:1037F6002DF582E43461F583E4F080040DBD80BECE
:10380600E49061ACF0FDEDFF7E00123D8D74AD2DB0
:0D381600F582E43461F583EFF00DBDFEE9AD
:013823002282
:023CC6008B2B46
:103CC800A2AF921EC2AF85A22C53A2FE8E838F8212
:103CD80005A28C838D827409122064E52B53A2FE01
:103CE80043A22012206653A2DF852CA2A21E92AF07
:013CF800FFCC
:013CF90022A8
:103DAA00A2AF921EC2AF8C838D82EF12206443A20F
:0C3DBA002012206653A2DFA21E92AFFF71
:013DC60022DA
:023D45008F26C7
:103D4700A2AF921EC2AFE4F5838D8274061220647F
:103D5700E52643A22012206653A2DFA21E92AF7F60
:013D6700015A
:013D68002238
:023D69008F26A3
:103D6B00A2AF921EC2AFE4F5838D82740A12206457
:103D7B00E52643A22012206653A2DFA21E92AF7F3C
:013D8B000136
:013D8C002214
:101E8D00A907E7FFA805EF93C3966008403B74FCD4
:101E9D002FFF80F00F08EF93C3966008402B74FB63
:101EAD002FFF80E00F08EF93C3966008401B74FA74
:101EBD002FFF80D00F08EF93D3966008400B74F975
:101ECD002FFF80C01F1F1F1F1FEF54FEF80303F7C6
:101EDD00E893FC08E893FD08E893FE08E893FF22D9
:101EED0009E993C39D6008402974FB29F980F10924
:101EFD00E993C39E6008401A74FA29F980E209E952
:101F0D0093D39F6008400B74F929F980D3191919DF
:101F1D001919E9C313C313FF22740093F8ECC39886
:101F2D004024701F740193F8EDC398401970147418
:0E1F3D000293F8EEC398400E7009740393F8F7
:101F4B00EFC39840037F00227F0122EDF8E6F008F3
:101F5B00A3DFFA22EDF8E0F608A3DFFA22E0A36391
:101F6B00A201F0A363A201DFF475A2002263A20118
:101F7B00F0A363A20122E0A363A201F0A363A20179
:101F8B00E0A363A201F0A363A201E463A201F0A3A7
:101F9B0063A201DFE175A20022E0A363A2016DFE43
:101FAB00936CFDEE058393FC158363A201DFEA7549
:101FBB00A200227F00E493A363A201F00F600CA3A5
:101FCB00E583C2E3F58363A20180EA75A20022E0F8
:101FDB00A363A201F0A3E583C2E3F58363A201DF50
:101FEB00EE75A20022E0A363A201F0A3E583C2E495
:101FFB00D2E3F58363A201DFEC75A20022E0A363B9
:10200B00A201F0A3E58344F8C2E5F58363A201DFE7
:10201B00EC75A20022E583C2E3F583E0A363A20182
:10202B00F0A363A201DFEE75A20022E583C2E4D226
:0A203B00E3F583E0A363A201F0A324
:1020450063A201DFEC75A20022E58344F8F583E085
:10205500A363A201F0A363A201DFEE75A20022F93A
:1020650022C002C004C00612FFF0D006D004D00280
:012075002248
:10001E00BF360BD217E4F545F546F561F562BF37ED
:04002E0002C21722D1
:10397B00C2A9438902906A27E0FFF58C8F8A75D91B
:10398B000475DA4875DB3175DC4975DD4975DE3157
:10399B00E4F5E9F5F9F5EBF5FB906A25E0601675B2
:1039AB00EC1075ED10E4F5FCF5FD755D08755B101D
:1039BB00755C01801375EC8075ED80E4F5FCF5FD0D
:0E39CB00755D80F55B755C10E4F5EEF5FE228F
:103BE300E4FEAF8CEFFD906A26E07003A3E06D6006
:103BF3000512397B7E01E5D920E2057E0212397B6D
:103C0300E58920E10512397B7E03D28C75D8407596
:083C1300B740D2AED2AFAF06FC
:013C1B002286
:030033000226BFE3
:0B26BF00C0E0C083C082C0D075D0080E
:1026CA00C2AF30DC56C3E5EC95EEC3955D5012E51A
:1026DA005C25ECF5EC30D70405FC801685FCFC8003
:1026EA0011C3E5EC955CF5EC30D70415FC80038545
:1026FA00FCFC301724854682854583E590F0054623
:10270A00E54670020545F582854583E5EEF0054606
:10271A00E5467002054553450FC2DC30D92930170A
:10272A0024854682854583E590F00546E546700294
:10273A000545F582854583E5EBF00546E5467002D9
:10274A00054553450FC2D930DA5DE55B700405FCD7
:10275A008010E55B25ECF5EC30D70405FC80038599
:10276A00FCFC301840E5475480F544E54725E0F580
:10277A0047309702054720160363470130270FE5C4
:10278A0047B56321755900755E00C2278017055E3B
:10279A00E55E5407700F535E3FE55E131313541F33
:1027AA002449F8A647C2DA30DB71E55B700405FDFF
:1027BA008010E55B25EDF5ED30D70405FD80038536
:1027CA00FDFDE55F655A6029E55A54077013E55A1D
:1027DA00131313541F2451F8E6F5482014036348D1
:1027EA00FFE548339296E54825E0F548055A535ADD
:1027FA003FB292301723854682854583E590F005DE
:10280A0046E54670020545F582854583E4F00546AE
:0D281A00E5467002054553450FC2DBD2AF05
:09282700D0D0D082D083D0E03281
:101988004241554400575F4D4F44454D00494E561E
:101998005F52454300494E565F5452414E530049E9
:1019A8004E565F414C4C004D4150424F415244000D
:1019B800554E49544D00003E2A2C312CCFE0F0E022
:1019C800ECE5F2F0FB20F1E8EDF5F0EEEDEDEEE3FD
:1019D800EE20EFEEF0F2E00A003E4C2C4230312CC3
:1019E800256C752CD1EAEEF0EEF1F2FC20EEE1EC7C
:1019F800E5EDE02C35302C3130302C3230302C33C2
:101A080030302C3630302C313230302C32343030CB
:101A18002C343830300A003E422C4731302C2562B5
:101A2800752CC8EDE2E5F0F1E8FF20EDE020EFF0DD
:101A3800E8B8ECE50A003E422C4731312C256275A6
:101A48002CC8EDE2E5F0F1E8FF20EDE020EFE5F04D
:101A5800E5E4E0F7E50A003E422C4730322C2562E7
:101A6800752CD3EFF0E0E2EBE5EDE8E520EFEEF2E0
:101A7800EEEAEEEC2020285254532D435453290A01
:101A8800003E532C4730332C256C752CC7E0E4E519
:101A9800F0E6EAE020F1F2E0F0F2E020EFE5F0E530
:101AA800E4E0F7E828ECF1290A003E532C473033EC
:101AB8002C256C752C202AE7E0E4E5F0E6EAE02026
:101AC800F1F2E0F0F2E020EFE5F0E5E4E0F7E828F5
:101AD800ECF1290A003E2A2C312CC0E4E0EFF2E5B3
:101AE800F020F1E8EDF5F0EEEDEDEEE3EE20EAE0C2
:101AF800EDE0EBE02E20CFF0EEF2EEEAEEEB20D2B6
:101B0800CC3531320A003E422C5430312C256275D6
:101B18002CC2FBE2EEE420D2D120EDE020F9E8F27D
:101B28000A003E422C5430322C2562752CD0E5E652
:101B3800E8EC20554E49544D0A003C21003C423007
:101B4800313D003C4731303D003C4731313D003CA0
:101B58004730323D003C4730333D003C5430313D46
:101B6800003C5430323D000ACEF8E8E1EAE020E4D7
:101B7800E0EDEDFBF5210A000ACEF8E8E1EAE02005
:101B8800F1E8EDF5F0EEEDE8E7E0F6E8E80A000A3E
:101B9800D6E8EAEB20D2C8D20A000AD6E8EAEB2057
:101BA800D2D10A000A2E2E2EE020E4EEEBE6E5ED77
:101BB80020E1FBF2FC20D2C8D2210A000A2E2E2EE8
:101BC800E020E4EEEBE6E5ED20E1FBF2FC20D2D1EB
:101BD800210A000AC3EEF2EEE220EFE0EAE5F22085
:101BE800EA20EEF2EFF0E0E2EAE50A00FF1988FFEA
:101BF800198DFF1995FF199DFF19A7FF19AFFF1937
:101C0800B8FF19BE0008040C020A060E0109050DEA
:041C1800030B070FA4
:103DCD0052668D00000000000000000000000000A1
:053DDD000000000000E1
:103E1900EF540F901C0C93FEC454F0FEEFC4540FE2
:043E2900932EFF22B3
:0100320022AB
:023AEC008F2E1B
:103AEE00906924E0FF04F074A02FF582E43466F5AB
:103AFE00837420F0E4FFEFC39D503BE52E75F00379
:103B0E00A424F4F582E4341BF583E493FB7401934F
:103B1E00FA740293F98F82758300121C35FE906938
:103B2E0024E024A0F582E43466F583EEF00F90696C
:063B3E0024E004F080C049
:013B4400225E
:103CFA00742D2FF582E43461F583E0FE64206016AA
:103D0A00906924E0FD04F074A02DF582E43466F590
:063D1A0083EEF00F80DAD9
:013D20002280
:10207600200B09AF267E007D03122E9BE490692477
:10208600F0F526E52675F003A424F4F582E4341B66
:10209600F583E493FB740193FA740293F9121C1C02
:1020A6007003022222E4F528F529F527742D252749
:1020B600F582E43461F583E0FF700302221DE52614
:1020C60075F003A424F4F582E4341BF583E493FB52
:1020D600740193FA740293F9852882758300121CA1
:1020E60035FEEFB506087529010528022218E529EF
:1020F6007003022218EE6003022213AD28AF2612E7
:102106003AECE526B40700400302221D902119F897
:1021160028287302212E0221C80221FD0222010273
:10212600220502220B02220FAF27123CFA742D253C
:1021360027F9E43461FA7B01C0031B8B3175320049
:10214600753300E4F534D0031222238F2D8E2C8DA7
:102156002B8C2AE4FFFEFDFCAB2DAA2CA92BA82A6A
:10216600C3121D3E6022AB2DAA2CA92BA82AE47F00
:10217600207E1CFDFC121C9E121D30906A26EEF07D
:10218600A3EFF0E4906A25F0E47FB07E04FDFCAB9B
:102196002DAA2CA92BA82AD3121D3E407A906A2577
:1021A6007401F0AB2DAA2CA92BA82A7F007EC2FDB4
:1021B6007C00121C9E121D30906A26EEF0A3EFF0F2
:1021C6008055AF27123CFAD21A742D2527F9E4342C
:1021D60061FA7B01C0031B8B31753200753300E455
:1021E600F534D0031222238F2D8E2C8D2B8C2A9022
:1021F600669FE52DF08020D216801CD2148018D25E
:1022060016D2148012D215800ED210800AE4F52957
:0C221600F52805270220B20526022089C9
:012222002299
:102CB2007BFF7A1979BF12138A906A25E0602FA3ED
:102CC200E0FEA3E0FFC3E49FFFE49EFEAB07FAE44D
:102CD200F9F8FF7EC27D01FC121C9E8F318E308D71
:102CE2002F8C2E7BFF7A1979E112138A802F906A3A
:102CF20026E0FEA3E0FFC3E49FFFE49EFEAB07FADB
:102D0200E4F9F87F207E1CFDFC121C9E8F318E3070
:102D12008D2F8C2E7BFF7A1979E112138A7BFF7A31
:102D22001A791FA216E433F52E12138A7BFF7A1A40
:102D3200793EA214E433F52E12138A7BFF7A1A79B4
:102D42005FA21AE433F52E12138A301A1F7BFF7A20
:102D52001A798990669FE075F00AA4FFAEF0E48FBD
:102D6200318E30F52FF52E12138A801D7BFF7A1AD1
:102D720079B290669FE075F00AA4FFAEF0E48F315D
:102D82008E30F52FF52E12138A7BFF7A1A79DD1217
:102D9200138A7BFF7A1B790EA215E433F52E1213E8
:102DA2008A7BFF7A1B792AA210E433F52E12138A4A
:012DB20022FE
:102830007E1B7F42123618EF4E70037F01227E1BF3
:102840007F45123618EF4E70030228D71239D990FF
:102850006A38121D4FE4FFFEFDFC906A38E0F8A3D1
:10286000E0F9A3E0FAA3E0FBC3121D3E6025906AE5
:1028700038E0F8A3E0A3E0A3E0E47F207E1CFDFCA9
:10288000121C9E121D30906A26EEF0A3EFF0E49029
:102890006A25F0E47FB07E04FDFC906A38E0F8A37E
:1028A000E0F9A3E0FAA3E0FBD3121D3E4038906AA2
:1028B000257401F0906A38E0F8A3E0A3E0A3E07F7C
:1028C000007EC27D017C00121C9E121D30906A2683
:1028D000EEF0A3EFF0800F906A2674FFF0A374B8B7
:1028E000F0E4906A25F07E1B7F4B123618EF4E60A5
:1028F0000C123DFFEF24D024FF92168002C2167EF8
:102900001B7F51123618EF4E600C123DFFEF24D0A2
:1029100024FF92148002C2147E1B7F57123618EFD8
:102920004E600C123DFFEF24D024FF921A8002C2A9
:102930001A7E1B7F5D123618EF4E60131239D9E4F0
:102940007B0AFAF9F8121C9E90669FEFF08005E46E
:1029500090669FF07E1B7F63123618EF4E600C125C
:102960003DFFEF24D024FF92158002C2157E1B7F0D
:1029700069123618EF4E600C123DFFEF24D024FF91
:0829800092108002C2107F00DA
:01298800222C
:103DE300906A2674FFF0A374B8F0E4906A25F01289
:0C3DF3002830EF600312207612397B228A
:103B450075637FC213D218C21DD227C21BC211C210
:103B55001CE49067E0F0906923F0FFEF25E024E195
:103B6500F582E43468AD82F5168D17F583E4F00F20
:103B7500BF20E8E4FFEF25E02425F582E43469ADB4
:103B850082F5168D17F583E4F00FBF80E8C291C268
:043B950090123BE36C
:013B99002209
:10389E00201069906379E0FE30E713541F25E02471
:1038AE00DFF582E43468AD82F5168D1780189063CB
:1038BE0079E0540F75F010A42415F582E5F0346903
:1038CE00AD82F5168D17E4FEEF24FBFDEEC39D5081
:1038DE002B851782851683E04480F0747A2EF5824C
:1038EE00E43463F583E0851782851683A3F07402B2
:0E38FE002517F517E43516F5160E80CCD21CF2
:01390C002298
:10328D00906923E004F024DF7003023337E0FF255B
:10329D00E024DFF582E43468AD82F5168D17F583F1
:1032AD00E060DD0513E513AC127002051214F58212
:1032BD008C83747FF0EF2480FF0513E513AC12703F
:1032CD0002051214F5828C83EFF08513828512832B
:1032DD00F030D003E0F4F00513E51370020512850C
:1032ED001782851683A3E0FF0513E513AC12700258
:1032FD00051214F5828C83EFF0851782851683A352
:10330D00E06455851382851283F020D012851782D3
:10331D00851683A3E0F46455851382851283F00529
:10332D0013E513700205127F0522E4906923F0FF67
:01333D00226D
:103121009067E0E004F024EF70030231D1E0FF7515
:10313100F010A42415F582E5F03469AD82F5168D01
:1031410017F583E060DA851382851283747FF005B9
:1031510013E51370020512EF2450FF8513828512C7
:1031610083F00513E51370020512F582851283EFD2
:10317100F030D003E0F4F0E4FF0513E5137002052D
:1031810012851782851683A3E0851382851283F049
:103191000513E51370020512851782851683A3E0D6
:1031A1006455851382851283F020D012851782859C
:1031B1001683A3E0F46455851382851283F07402AB
:1031C1002517F517E43516F5160FBF08AC7F132246
:0631D100E49067E0F0FF4E
:0131D70022D5
:10298900201D03022AA4E4906475F03010179067A3
:10299900A0E054F0FFBF50047F2180027F059064BE
:1029A90076EFF080159067A0E054F0FFBF50047FE8
:1029B9000980027F02906476EFF090667AE0906475
:1029C90077F0301006A37414F080069064787401CF
:1029D900F0201003022A78E4906479F0906476E09C
:1029E900D3940540679067A0E0540FFF1475F00871
:1029F900A4FF7D057E01EED394084003022A9FAC13
:102A0900050D74752CF582E43464F5837450F0ACCB
:102A1900050D74752CF582E43464F583EFF0AC058B
:102A29000D74752CF582E43464F583E4F074A02EFA
:102A3900F582E43467F583E0FCAB050D74752BF57D
:102A490082E43464F583ECF00E0F80AA90647A7402
:102A590010F09067A0E0541F1490647BF0E4A3F099
:102A69009067A1E0FF123E1990647DEFF08027E4A2
:102A7900FD906476E0FFEDC39F501B74A02DF58295
:102A8900E43467F583E0FF74792DF582E43464F565
:0D2A990083EFF00D80DBC21D7F01227F0066
:012AA600220D
:103C1C00300D0B7E1B7F6FE4FBFDFC122AA7906618
:103C2C0097E0FCA3E0FDA3E0FEA3E0FFE4FAF9F8C3
:103C3C00EF2401FFEA3EFEE93DFDE83CFC9066976F
:093C4C00121D4FA212B3921222C4
:103C5500300D0B7E1B7F80E4FBFDFC122AA79066CE
:103C650097E0FCA3E0FDA3E0FEA3E0FFE4FAF9F88A
:103C7500EF2401FFEA3EFEE93DFDE83CFC90669736
:093C8500121D4FA212B39212228B
:1016840030172DC3E5469562FFE5459561FED3EF1E
:101694009440EE940040197B087D40AF62AE611225
:1016A4002F7CE5622440FFE43561540FF5618F62BD
:1016B400201960301341E55E543865596027E559B7
:1016C40024085438F559131313541F2449F8E6FF1A
:1016D4000511E511AC107002051014F5828C83EF2E
:1016E400F0151A80D1E51A600302189AD227D2198C
:1016F400C213C29102189A30270302189AD291D2C7
:1017040013751A04301203751A127510677511E1F6
:1017140002189A300D1F30120F7E1B7F977C677D55
:10172400E17B12122AA7800D7E1B7FA27C677DE1DC
:101734007B04122AA7C2199067E1E0F030D00FA30E
:10174400E0F4FF9067E1E06F6014123C1C229067A4
:10175400E2E0FF9067E1E06F6004123C1C229067B6
:10176400E1E054F0FFBF50047F0880027F018F2620
:10177400A212E433FFE526B401047E0180027E0058
:10178400EE5F6012300D0B7E1B7FACE4FBFDFC12A0
:101794002AA7123C55222012047F0180027F00E513
:1017A40026B408047E0180027E00EE5F6012300DD4
:1017B4000B7E1B7FC4E4FBFDFC122AA7123C5522BE
:1017C400E4F527E527C395265061E52725E024E3C2
:1017D400F582E43467F583E0F020D025E52725E0A1
:1017E40024E4F582E43467F583E0F46455FFE527E7
:1017F40025E024E3F582E43467F583E0B50724802B
:1018040026E52725E024E4F582E43467F583E064E3
:1018140055FFE52725E024E3F582E43467F583E00A
:101824006F6004123C1C2205278098E4F527E52606
:101834002401FFE433FEC3E5279FEE6480F874803F
:10184400985020E52725E024E1F582E43467F58308
:10185400E0FF74A02527F582E43467F583EFF005F3
:101864002780CBD21D90668FE0FCA3E0FDA3E0FEB1
:10187400A3E0FFE4FAF9F8EF2401FFEA3EFEE93DB4
:10188400FDE83CFC90668F121D4FE526B40103D39E
:101894008001C3921222301B7AE55F655A6048E5E5
:1018A4005F24085438FFE55A54386F60047E018081
:1018B400027E00E51B60047D0180027D00EE5D7008
:1018C400030219870513E513AC127002051214F50F
:1018D400828C83E0FEE55F131313541F2451F8A692
:1018E400068F5F151B80B8C290C21BC2119066930D
:1018F400E0FCA3E0FDA3E0FEA3E0FFE4FAF9F8EFC7
:101904002401FFEA3EFEE93DFDE83CFC90669312AB
:101914001D4F22E4F51B75126875136112328D8F09
:101924001BE51B700512328D8F1B1231218F26E5AA
:101934002670051231218F26E526251BF51B641818
:101944007041300D0D7E1B7FDB7C687D617B18123E
:101954002AA77512687513610513E513AE12700298
:10196400051214F5828E83E0FFE55F131313541FF1
:101974002451F8A607E55F24085438F55F151BD2F7
:031984001BD290E3
:01198700223D
:0B3E4800301C05C21C7F01227F0022FD
:1031D800E4FF0F2405F582E43461F5837408F00FE9
:1031E80074052401F582E43461F583E4F07C667D9E
:1031F80092FEED1DAA0470011CF5828A83E0FBAAE9
:10320800070F74052AF582E43461F583EBF00EBEEE
:1032180004E07C667D96E4FEED1DAA0470011CF5B1
:10322800828A83E0FBAA070F74052AF582E43461D9
:10323800F583EBF00EBE04E07C667D9AE4FEED1D9E
:10324800AA0470011CF5828A83E0FBAA070F7405A3
:103258002AF582E43461F583EBF00EBE04E07C6667
:103268007D9EE4FEED1DAA0470011CF5828A83E0B0
:10327800FBAA070F74052AF582E43461F583EBF0A5
:043288000EBE04E092
:01328C00221F
:033E5300C2AE22DA
:10348A00020879E493A3F8E493A34003F68001F2D7
:10349A0008DFF48029E493A3F85407240CC8C33343
:1034AA00C4540F4420C8834004F456800146F6DF12
:1034BA00E4800B0102040810204080903DC7E47E9E
:1034CA00019360BCA3FF543F30E509541FFEE49307
:1034DA00A360010ECF54C025E060A840B8E493A3CE
:1034EA00FAE493A3F8E493A3C8C582C8CAC583CAF9
:1034FA00F0A3C8C582C8CAC583CADFE9DEE780BEB1
:013DE20000E0
:101C1C00BB010689828A83E0225002E722BBFE02C6
:091C2C00E32289828A83E49322F9
:101C3500BB010CE58229F582E5833AF583E0225064
:101C450006E92582F8E622BBFE06E92582F8E222AE
:0D1C5500E58229F582E5833AF583E49322C8
:101C620075F008758200EF2FFFEE33FECD33CDCC39
:101C720033CCC58233C5829BED9AEC99E5829840BC
:101C82000CF582EE9BFEED9AFDEC99FC0FD5F0D699
:101C9200E4CEFBE4CDFAE4CCF9A88222B800C1B9C3
:101CA2000059BA002DEC8BF084CFCECDFCE5F0CB01
:101CB200F97818EF2FFFEE33FEED33FDEC33FCEB3A
:101CC20033FB10D703994004EB99FB0FD8E5E4F9F5
:101CD200FA227818EF2FFFEE33FEED33FDEC33FCE2
:101CE200C933C910D7059BE99A4007EC9BFCE99AD6
:101CF200F90FD8E0E4C9FAE4CCFB2275F010EF2F1B
:101D0200FFEE33FEED33FDCC33CCC833C810D7071A
:101D12009BEC9AE899400AED9BFDEC9AFCE899F855
:0E1D22000FD5F0DAE4CDFBE4CCFAE4C8F922E8
:0E1D3000C3E49FFFE49EFEE49DFDE49CFC22C4
:101D3E00EB9FF5F0EA9E42F0E99D42F0E89C45F0FB
:011D4E002272
:0C1D4F00ECF0A3EDF0A3EEF0A3EFF02207
:101D5B00A8828583F0D083D082121D72121D72125D
:101D6B001D72121D72E473E493A3C583C5F0C58382
:101D7B00C8C582C8F0A3C583C5F0C583C8C582C8D2
:011D8B002235
:10132800E53A242EF8E6053A22782B302502782E65
:10133800E475F001121DED021C1C201EEB7F2ED25D
:101348001E8018EF540F2490D43440D4FF30220B61
:10135800EF24BFB41A0050032461FFE53B60021577
:101368003B053EE53E7002053D30250D782BE475C2
:10137800F001121DEDEF021D8C023B9A7403D22579
:101388008003E4C225F53A8B2B8A2C892DE4F53BA2
:10139800F53DF53EE53B60077F2012136380F57548
:1013A8003CFFC21FC21EC220C221C223C224C226C1
:1013B800121331FF700D3025057F00121374AF3EF4
:1013C800AE3D22B4255FC2D5C222121331FF24D00C
:1013D800B40A00501A75F00A783B30D50508B6FFF4
:1013E8000106C6A426F620D5047002D22180D9248D
:1013F800CFB41A00EF5004C2E5D222021574D21FEE
:1014080080C6D21E80C0D22080BCD2D580BAD2235A
:1014180080B47F201213632020077401B53B00407D
:10142800F1121328FF12136302139CD226D22480D0
:1014380095121328FB121328FA121328F94A4B7035
:101448000679457A167BFF20202EE53B602A7E0030
:101458008E82758300121C3560060EEE653C70F0B6
:10146800C2D5EBC0E0EAC0E0E9C0E0EE1215BBD09F
:10147800E0F9D0E0FAD0E0FB121C1CFF60AAEBC038
:10148800E0EAC0E0E9C0E0121363D0E02401F9D03B
:10149800E03400FAD0E0FBE53C0460DCD53CD980C0
:1014A800877BFF7A1579B7D220809C7910800279E2
:1014B80008C224C2268008D2D5790A8004790AC2D3
:1014C800D5E53C047002F53CE4FAFDFEFF12132852
:1014D800FC7B08201F13121328FD7B10301E0A12F4
:1014E8001328FE121328FF7B20EC3382D592D550A7
:1014F80013C3E4301E069FFFE49EFEE4201F039DF5
:10150800FDE49CFCE4CBF8C21FEC700CCFCECDCC34
:10151800E824F8F870F38017C3EF33FFEE33FEEDDD
:1015280033FDEC33FCEB33FB994002FB0FD8E9EBBE
:10153800301F05F8D0E0C448B21FC0E00AEC4D4E99
:101548004F78207B0070C2EAB53C0040BCC0E01276
:1015580015BDD0F0D0E0201F04C4C0E0C4B21FC045
:10156800F012134CD0F0D5F0EB02139C121E4C1461
:10157800395314B358140A4C14064214B74F14BF05
:0F1588004414BF49141F4314C55514A94614A990
:101597004514A947166550140E2D14122E14352B19
:1015A700141623143320164E2A13CE480000142D88
:1015B7003F3F3F00790AA2D5202114302309B910F3
:1015C700020404B9080104A2D52024025001042012
:1015D70020689220B53B005034C0E07F20302119AD
:1015E7007F30A22072247223500F121614C220C219
:1015F70024C223C2267F30800F302303E9C0E012C4
:101607001363302303D0E0F9D0E0B53BCC30231788
:101617007F30B9100C1213637F583022077F788010
:1016270003B908031213633020057F2D0213637F6C
:10163700202026F87F2B2024F322922080CF286EAB
:10164700756C6C2900D21F121328301FF8C21F783F
:101657003B30D50108F60213CE2D504349581213DB
:10166700282403B405004001E49016609312135434
:0D167700743A121354D221753B040214B3CF
:102223008B2E8A2F8930E4F53AF539F538F537F5F1
:1022330035F536E532453345316012EBC0E0EAC08F
:10224300E0E9C0E0AB31AA32A933121DFDAB2E0584
:1022530030E530AA2F7002052F14F9121C1CF53B30
:10226300C394094007E53BD3940D40E1E53B64206B
:1022730060DBE53BB42D054336038016E53BB42B09
:1022830005433601800C74FF2530F53074FF352F7C
:10229300F52FE53460046410703FAB2EAA2FA930EC
:1022A300121C1C64306009E534702E75340A8029D1
:1022B300900001121C35FF64786004EFB458134397
:1022C300360175341074022530F530E4352FF52FBF
:1022D3008007E5347003753408AB2E0530E530AA6A
:1022E3002F7002052F14F9121C1CF53BC394614097
:1022F3000AE53BD3947A5003533BDF74D0253BF577
:102303003BC3940A400CE53B9411406D74F9253BA3
:10231300F53BE53BD395345060433601853A3F8521
:10232300393E85383D85373CAF347E00E4FCFDAB58
:102333003AAA39A938A837121D9EC8ECC8C9EDC9F5
:10234300CAEECACBEFCBE4FCFDFEEB253BF53AEE40
:102353003AF539ED39F538EC38F537AF3AAE39ADF2
:1023630038FCAB3FAA3EA93DA83CD3121D3E500307
:102373000222DC4336040222DCE53620E003E4805B
:102383002DE53245334531601EAB2EE53024FFF990
:10239300E52F34FFFAEBC0E0EAC0E0E9C0E0AB317F
:1023A300AA32A933121DFDE53630E20774FFFFFEA2
:1023B300FDFC22E536AF3AAE39AD38AC3730E10338
:0423C300021D3022A5
:101D8C00BB010689828A83F0225002F722BBFE0136
:021D9C00F32230
:101D9E00E88FF0A4CC8BF0A42CFCE98EF0A42CFCE4
:101DAE008AF0EDA42CFCEA8EF0A4CDA8F08BF0A462
:101DBE002DCC3825F0FDE98FF0A42CCD35F0FCEBC1
:101DCE008EF0A4FEA9F0EB8FF0A4CFC5F02ECD3986
:0F1DDE00FEE43CFCEAA42DCE35F0FDE43CFC22F3
:101DED00FAE6FB0808E6F925F0F618E6CA3AF622F7
:101DFD00BB011A89828A83D0F0D0E0F8D0E0F9D007
:101E0D00E0FAD0E0FBE8C0E0C0F0021E7B5016E91E
:101E1D00F8D083D082D0E0F9D0E0FAD0E0FBC082D8
:101E2D00C083021E72BBFE16E9F8D083D082D0E0CB
:0F1E3D00F9D0E0FAD0E0FBC082C083021E8422FD
:101E4C00D083D082F8E4937012740193700DA3A325
:101E5C0093F8740193F5828883E473740293686039
:061E6C00EFA3A3A380DF39
:091E7200EBF608EAF608E9F62295
:091E7B00EBF0A3EAF0A3E9F02268
:091E8400EBF208EAF208E9F2228F
:00000001FF
